:030000000219FDE5
:03000B000200AA46
:03002B000201656A
:03005B000202FBA3
:030073000202E1A5
:1000800002030406080C10182030406080040608A3
:100090000C10182030406080A0C000070F1F3F0DDB
:1000A0000D0403060D0503030202C2AFC0D0C0E079
:1000B000206217E5256002E473E525F4F58A758B67
:1000C00000D262D0E0D0D0D2AF3285268AC262E5BB
:1000D00026F46035306803207210758B00D0E0D0B4
:1000E000D0D297D295D293D2AF32D297D295D29323
:1000F000206E0C206609740AD5E0FDE57E429075FD
:100100008B00D0E0D0D0D2AF32758A00C28DD262DF
:1001100001FF01B9306805206602C29701B9306855
:1001200005206602C29501B9306805206602C293B7
:1001300001B9C29630680A2066077408D5E0FDC28E
:100140009701B9C29430680A2066077408D5E0FDAB
:10015000C29501B9C29230680A2066077408D5E0DA
:10016000FDC29301B9C2AFC2AD53E6EFC0D0C0E04B
:10017000D2D3D2AFC2CEE52A6007207449152A2116
:10018000C67800790020742EE580307E01F430E5D9
:100190000278FF53DACF207E0343DA20307E034318
:1001A000DA10C2D8C271E580307E01F430E5027900
:1001B000FFC3E89970CB306103752A402074037542
:1001C0002A40885FD27020740DE52B6004152B2126
:1001D000D643DA01C2D820700221E9A85F2061026B
:1001E000C27020740221E788227882B60403852237
:1001F00024C3E52594404002D26420CF0AD0E0D049
:10020000D043E610D2AD32C2CF053A7802E52A607B
:1002100005307402152AC3E55F940140057562003C
:100220004133756300756C00E5622401F56250038B
:100230007562FF7982B7020D306D1DC3E5229432DD
:100240004016854D227982B7030E306D0BC3E5222F
:1002500094324004798E8722C3E5239522600840BA
:1002600004152341670523D8CA056CE56C70021597
:100270006CD56D63756D017805C3E56C956E40575F
:10028000C3E56C956F50087801756D0302029BC33E
:10029000E56C957050057801756D01C3E565952491
:1002A000401E7982B7040241CC206D14852465E597
:1002B0006C046003856E6C756D0175233C0202D77A
:1002C000E5652850057565FF41CCF565E565047069
:1002D000067563FF756CFFD0E0D0D043E610D2AD59
:1002E00032C2AFC0D053E67FC2607591008556948C
:1002F000855795759104D0D0D2AF32C2AF53E6EF97
:10030000C2ADC0D0C0E0C0F0D2D3D2AFA8FBA9FC30
:10031000C2D8307102616253DACF207E0343DA1013
:10032000307E0343DA20D271E580307E01F420E58F
:1003300002613988278928A14153DACF207E0343FF
:10034000DA20307E0343DA10C2D8C271307402A1C1
:100350002D7800E580307E01F430E502A12D885F24
:10036000A11553DACF207E0343DA20307E0343DA2F
:1003700010C271206102813B53DACF207E0343DA41
:1003800010307E0343DA20C2D8D271885A895BC309
:10039000E89558F8E99559F97B007E087A00C3E89A
:1003A000948CE994005005755E00812D882178A217
:1003B000E6A8216055C3E894C8E994005008E4D247
:1003C000E4FB7A0A8108C3E89468E994015008E4E0
:1003D000D2E3FB7A0F8108C3E894D0E99402500875
:1003E000E4D2E2FB7A1E8108C3E894A0E9940550A8
:1003F00008E4D2E1FB7A3C8108C3E89498E99408C8
:100400005008E4D2E0FB7A787E00C3E8955CFCE912
:10041000955DFD30E70AECF42401FCEDF43400FDB9
:10042000755E00C3EC9AED9E5003755E01885C8991
:100430005D855A58855B597802A115C3E89527F860
:10044000E99528F9307C0281F9307B0281F9307A14
:100450000281F2207502815EE9FDE8FC817DE9C33D
:1004600013F9E813F830790281F2E9C313F9E813BC
:0D047000F830780281F2E9C313FDE813FCB7
:10047D00206126C3EC941CED940240028194ED7032
:10048D0018C3EC94C850120529C3E529940A5002EB
:10049D00A12D755F00D270A12DE52960021529747B
:1004AD0000207F037896E624FAFEE43400FFC3ECC7
:1004BD009EFCED9FFD50067800790081F9C3EC9408
:1004CD00FFED9400400678FF790081F9EC8575F019
:1004DD00A4C5F0A2F733F87900400302051578FFA3
:1004ED007900020515E9C313F9E813F8307C0EE91C
:1004FD00600278FFC3E81338F8E43400F9C3E894D8
:10050D00FFE99400400278FF885FD270206102A15C
:10051D002D741FF4552F4BF52FC274EB7002D2744E
:10052D00752A40307403752A0A306102A141207486
:10053D000353DAFE207403752B20D0F0D0E0D0D019
:10054D00D2AD43E6103279010205717903020571CE
:10055D00790A020571791E020571796402057179B6
:10056D00C80205717817E4D5E0FDD8FAD9F6227ADC
:10057D00147B780205987A107B8C0205987A0D7B96
:10058D00B40205987A0B7BC80205987902B27DE416
:10059D00C294D5E0FDC295D5E0FDD295D5E0FDD252
:1005AD0094D5E0FDC297E576D5E0FDD2977496D54A
:1005BD00E0FDD9D9EAF8D5E0FDD8FBDBCEC2942217
:1005CD00C37C007D0075F00005F0EA33FAEB33FBD8
:1005DD0050F6EB13FBEA13FAC3E9FFE8FEE89AF8CD
:1005ED00E99BF95004EFF9EEF8B3EC33FCED33FD74
:1005FD00D5F0DFEDF9ECF822E889F08A20D2D4F8B5
:10060D00A9F07B0030F70B7BFFF42401F8E9F434FB
:10061D0000F9E88520F0A4ADF0F8E98520F0A4AF4D
:10062D00F0FEED2EF974003FFA7C04C3EA13FAE9EB
:10063D0013F9E813F8DCF48BF030F70AE8F4240131
:10064D00F8E9F43400F9E889F0C2D4F8A9F0227879
:10065D0082B604030206FBC3E55F9419401EE52D27
:10066D0054067018206D3678057994E71460077874
:10067D000A1460027812C3E54198401F306D098558
:10068D006765756CFF756D01852224E4F545F546AA
:10069D00F547F548F549C26D0206FBD26D7994E731
:1006AD00147013E523F43333F913F8E9540104F905
:1006BD00E854FE0206EFE714147014E523F4333307
:1006CD0033F913F8E9540304F9E854FC0206F7E58D
:1006DD0023F433333333F913F8E954070404F9E8F9
:1006ED0054F8C39440F8E99400F98845894622C32B
:1006FD00E54113F9E54013F8C3E54598F8E546994A
:10070D00F9500CC3E89480E994FF4016020733C3F7
:10071D00E8947FE994005003020733787F79000253
:10072D000733788079FF884A894B22E54A2547F8B7
:10073D00E54B3548F9854B20E4300701F43549FA8E
:10074D0030E709C3EA94F04015020771C3EA940F2C
:10075D00500302077178FF79FF7A0F020771780055
:10076D0079007AF0C3E5249564500AC37401952489
:10077D00500B02078FE54B20E70E02078FE54B303C
:10078D00E706884789488A492278A4E6FAC3E54AEC
:10079D0033F8E54B33F9D105E930E70BC3E8948025
:1007AD00E994FF4013E1C9C3E8947FE99400500236
:1007BD00E1C9787F7900E1C9788079FFE820E715F4
:1007CD00C3E52398F84009C3E8940140030207F0FC
:1007DD0078010207F0E8F424012523F8400302070D
:1007ED00F078FF884C2278A5E6FAA848A949D105EA
:1007FD00E930E70CC3E89401E994FF4016020824A0
:10080D00C3E894FFE99400500302082478FF7900AF
:10081D00020824780179FFE920E715C3E54C98F823
:10082D004009C3E89401400302084B780102084BCC
:10083D00E8F42401254CF8400302084B78FF882486
:10084D002278FFC26420693D206A12D264C3E5415B
:10085D00940A4009C3E52594405002C26479A1E78A
:0F086D006023E541601F74FF8541F0848539F0F9
:10087C00306A0375F005A4F8C5F0600278FFC3E890
:10088C0095675002A867886622C3E5409440E5410D
:10089C009401E56650031401A6046002F566227803
:1008AC0083E6F520120F4475E89012055375E89015
:1008BC00E5E820ECFBA8BDA9BE120FDE75715575DD
:1008CC007200C3740013FD7455606613FC74552CD0
:1008DC00FC74003DFDECFAEDFBC3E89AE99B401477
:1008EC00E5712455F571E5723400F572EA2CFAEBDA
:1008FC003DFB80E5AE71AF72C3E57213F9E5711380
:10090C00F8C3E913F9E813F87A03C3E913F9E81308
:10091C00F8DAF7AA201A70097571007572000209CD
:10092C003D1AEA6008EE28FEEF39FFDAF88E718F77
:10093C00722275E890227883E6FFE5E820ECF7A8B0
:10094C00BDA9BE0573C3E57394084052757300E9E5
:10095C00FA79A0E76044EA7007E574601B02097835
:10096C00C3E895746010E5745006600C1402098499
:10097C000460F9020984E574F574C3946D401B7529
:10098C0064C0C394044013756480C39404400B7515
:10099C006440C39404400375640075BB0822EFC324
:1009AC009401601F7455601BC3E894FFE9940350D5
:1009BC0012C3E89571E995725009E564600C1564F1
:1009CC000209D6E564F460020564A864C3E52498C2
:1009DC005002A824C3E89565400AA865E565F46053
:1009EC000385656488258826E573B4070375BB10F9
:1009FC0022743279A687F0A4C5F0A2F733F8C3E8C5
:100A0C0095644002A86488228824882588268867F3
:100A1C00227540007541F022C2AF75C820A8CCA940
:100A2C00CDAA3A30CF010A75C824D2AFAB3BAC3C4F
:100A3C00883B893CC3E89BF8E99C206908F930673E
:100A4C000261394196AD3D8A3DF9EA9DFA60047820
:100A5C00FF79FFAE3EAF3F8B3E8C3FC3EC9FFCC398
:100A6C00E99CF542A83BA93CC3E89EF8E99FF9C371
:100A7C00E54113FBE54013FAE82AF540E93BF54163
:100A8C0050067540FF7541FF41E0AA40AB41AC40B8
:100A9C00AD417E047F02C3EB940440021E1FC3EBE6
:100AAC00940840021E1FC3ED13FDEC13FCDEF7C3CC
:100ABC00EA9CFAEB9DFBEF6009C3E913F9E813F824
:100ACC00DFF7EA28FAEB39FB8A408B4150067BFFB3
:100ADC008B408B41C3EB94025002D2673069047F88
:100AEC0003610B7892E6FFC3E537948240110FC384
:100AFC00E53794A040010FC3EF940640027F057EBA
:100B0C0005E541C4540FF9E541C454F0F8E540C47F
:100B1C00540F28F8C3E89EFAE99400FB4009C3EA95
:100B2C009402EB940050047A02E4FB6185AA40AB7A
:100B3C0041EBC4FEEAC4540F4EFCC3EA9CFAEB949E
:100B4C0000FBC3E813C313F8EA28FAEB3400FB8A62
:100B5C00408B41C3EB94024002C2677805EBC4FEA4
:100B6C007B00EAC4540F4EFAC3EA98FA4005C394CA
:100B7C000250027A027892E6FF306002618585525B
:100B8C0056855357D26043E680C3E49AF8E49BF948
:100B9C00306702811FE8FAE9FBD3E913FDE813FC87
:100BAC0088528953C3EF94036038EF20E00DE82C92
:100BBC00F8E93DF9ECFAEDFB020BDAE828F8E93933
:100BCC00F9C3E82402F8E93400F97AFE7BFFC3EF9D
:100BDC009403400E8A548B55884E894F8C508D51FE
:100BEC008153885489558A4E8B4F8C508D51306966
:100BFC0020C3E53394034019E542A2E713F8E55509
:100C0C00F4240138400B20E7087554FFF42401F557
:100C1C00558153E8FAD3E813FC8852C3EF94036070
:100C2C0020EF20E007E82CF8ECFA813FE8282402BA
:100C3C00F87AFEC3EF940340088A54884E8C508196
:100C4C005388548A4E8C50E56BC3335002646BF559
:100C5C006B306002815D753402D26043E680E52D15
:0F0C6C0054066026A840A941C3E913F9E813F81C
:100C7B00C2AF53E67F759100C3E498F594E499F500
:100C8B0095759104D26043E680D2AF22D26575444C
:100C9B0000752000306B03752040020CB6D26575D1
:100CAB004400752040306B03752000D2AF780120D3
:100CBB006722E52D54066002C265C3E541940540E9
:100CCB0013780294054008780394054002780630A7
:100CDB006902780A206019E544601530690AC3E59A
:100CEB003394034003D53406D2AFD26CA187916500
:100CFB00D2AF0000C2AF206726E541C3FB940F4083
:100D0B00027B0FEB240530730123306A0274282019
:100D1B00620123F93069027982E58BC39940B505ED
:100D2B0044E59B5440B52002A17130690A08C3E821
:100D3B00940A40010881DF20650281B6C26553E643
:100D4B007F7591003067107594007595FE75910451
:100D5B00D26043E68081B6AE40AF41C3E49EF594CA
:100D6B00E49FF595A158C3E5339402500281B63048
:100D7B00650281B6D802A18581DFC26C53E67F750F
:100D8B009100855494855595759104854E56854FE4
:100D9B0057D26043E680D2AFE52D54066008206A37
:100DAB00020533020DC1306C0D206B0A206507154F
:100DBB0081158102161622780030640530650278A1
:100DCB0001E53775F007A4F9E5F028F5F0E9A2F095
:100DDB0013A2F113A2F213F537C3947850037537AE
:100DEB0078C3E53795384008D266D297D295D2931F
:100DFB00306002A1FB855056855157D26043E68087
:100E0B0022207D11C2AF754302C294D296D2AF7528
:100E1B009F10020FDBC2AF754302C294D292D2AFC6
:100E2B00759F10020FDB307243207D20C2AF7543DC
:100E3B0003900143757E10D293C292306204C29527
:100E4B00C14FD294D2AF759F13020FDBC2AF754364
:100E5B0003900143757E10D297C296306204C295FF
:100E6B00C16FD294D2AF759F11020FDB207D17C2D9
:100E7B00AF75430390011ED293306202C295D2AF7D
:100E8B00759F13020FDBC2AF75430390011ED29700
:100E9B00306202C295D2AF759F11020FDB207D111C
:100EAB00C2AF754304C296D292D2AF759F11020F97
:100EBB00DBC2AF754304C292D296D2AF759F1302B9
:100ECB000FDB307243207D20C2AF7543059001329A
:100EDB00757E40D295C294306204C297C1EBD29614
:100EEB00D2AF759F10020FDBC2AF75430590015453
:100EFB00757E04D295C294306204C293E10BD292F8
:100F0B00D2AF759F10020FDB207D17C2AF75430563
:100F1B00900114D295306202C297D2AF759F100226
:100F2B000FDBC2AF754305900128D2953062EBC23F
:100F3B0093D2AF759F10020FDB207D11C2AF7543AB
:100F4B0006C292D294D2AF759F13020FDBC2AF755C
:100F5B004306C296D294D2AF759F11020FDB30724B
:100F6B0042207D20C2AF754301900154757E04D29F
:100F7B0097C296306204C293E187D292D2AF759F2B
:100F8B0011020FDBC2AF754301900132757E40D267
:100F9B0093C292306204C297E1A7D296D2AF759FEB
:100FAB0013E1DB207D16C2AF754301900128D29768
:100FBB00306202C293D2AF759F11E1DBC2AF7543B2
:100FCB0001900114D293306202C297D2AF759F1376
:100FDB00C26622900112757E00D297D295D293C22F
:100FEB0096C294C292C2622278807607087607086E
:100FFB0076010876040876FF0876FF08760A0876ED
:10100B0002087601087601788C760108760008765E
:10101B00B40876FF0876FF0876FF0876030876FF9C
:10102B000876010876FF0876250876D008767808CA
:10103B0076C80876040876FF0876010876000876ED
:10104B007A08760A0876010876010876000876FF9A
:10105B00227887E6FFC272BF0302D2727888C27D04
:0E106B00E630E102D27DC27E7889E630E102F5
:10107900D27EC3EF94026008758E01D27302108E7E
:10108900758E00C273227880E6149000809378A44C
:10109900F67881E6149000809378A5F67886E614B0
:1010A90090008D9378A6F6789FE6F8700108C3E85A
:1010B900941140027811E82828F56E256E256E28CE
:1010C900F56F256E2828F570789CE67538FF753917
:1010D9000CB402067538A075390AB403067538824E
:1010E90075390578A3E61490009A93F569120FDE15
:1010F90022227896E6FA7897E6FB7888E6B4030523
:10110900C3EB940EFB307F047A007BFFC3EB9AFCA0
:10111900C3948250027C827575000575EC8575F063
:10112900A4C3E5F0947D40F222D27F11FB1205623F
:101139007A007B007C10120558E55F2AFA74003B9F
:10114900FBDCF37C04C3EB13FBEA13FADCF7FEC206
:101159007F11FB22E5EF20E6037520000520903F73
:10116900FFE520146006901DFF14600093046003DE
:1011790075EF1253D9BF7581C043FF8012055375AE
:10118900EF0243B203E5B3240420E70DF521E5E3BB
:1011990020E0068521B343E301120FDE7580FF7558
:1011A900A40075F1B275D4DF7590A975A5FC75F227
:1011B900FC75D50175A60175E241E4F8F6D8FD750F
:1011C9006B01120FF312165E78988676753001C29C
:1011D900AF12056C12057C120562120583120562B5
:1011E90012058A12056212178112056C12056C121A
:1011F9000567C2AF78FA79FA308507D9FBD8F702C3
:101209001C00115C118F11FA11FB78988676120F68
:10121900DE75885075891275C82475910475D84092
:1012290075A82275B80275E690759B80759D007545
:10123900D10E75BC5875BB0875BA1175E8801205D1
:1012490053D2AF1208AB53DACF207E0343DA2030F2
:101259007E0343DA1043DA01C2D8C27112056CD297
:10126900617B037A0CE55E70077A0CDB030211FBE4
:101279001205622070030211FBC270E55FC394027C
:1012890040E1E52F541F856160F561B560D5DAD578
:10129900C26153DACF207E0343DA20307E0343DA7A
:1012A90010C2D8C27178A2E67008D274E52F54E052
:1012B900F52FC275752900120567307409C3E52930
:1012C900940A4002D27512055878023074027800E7
:1012D900C3E55F9840F0C2AF12057C12057C120588
:1012E9007CD2AF12056C754D00120558788CE6C397
:1012F900940150030213C8E530C39401500302134B
:10130900C8207435C3E55F94FF50030213C8C2AF08
:10131900120591D2AF120567C3E55F940150EFC280
:10132900AF12057C12055D12057CD2AF120567C3A9
:10133900E55F94FF40E90218067F05D27F11FB1291
:101349000567C2AFC27F11FBAE5FC3E55F947FD271
:10135900AF4076120553C2AF120591D2AFDFDC312F
:1013690032C3EE94057897F612056C1216A012177F
:10137900897F0AD27F11FB120567C2AFC27F11FBB9
:10138900AE5FC3E55F947FD2AF50E6120553C2AF9B
:1013990012057C12055D12057CD2AFDFD63132EE23
:1013A90024057896F612056C1216A01217B81205C4
:1013B9006711FBC3E55F94FF5002610A021806C377
:1013C900E55F954D4003855F4D1205677801798882
:1013D900E7B403027805C3E55F98400241F2C2AF62
:1013E900120591120591120591D2AF12056C753053
:1013F90000E4F531F5320531E531F470390532781B
:101409009AE67819146012783214600D787D1460A8
:101419000878FA146003753200C3E532984017154D
:10142900327531B478998676C2AF120591D2AF7808
:1014390098867612056712055DE52A7005307402F3
:1014490021FB78012074027806C3E55F9840A71252
:101459000567E52A70030211FBC2AF120FDEE4F53E
:0F14690022F523F524F525F526F56AD2AF78850F
:10147800E6C333F568E4F545F546F547F548F5491B
:10148800F573F52CF52DF53775730875BB10120536
:101498005312093EE5E820ECFBA8BDA9BEE970019E
:1014A800F8887412094275730875BB107887E6FED0
:1014B8007602115C7887EEF6C2AF7564FF1209FDFB
:1014C800852264852265852266D2AF75220175243E
:1014D8000175250175260185636C756D017888E6AF
:1014E800B40307C27D307602D27DD268D2697533E3
:1014F80000120F44120F69120A1D120A24120A1D43
:10150800120A24120A1D02151DC2AF115CD2AF7552
:10151800730075BB08120CA812065C120DC2120EDD
:101528000C120A24120C97306D031206FC20670374
:1015380012084E306703120895120DC2120E3112AE
:101548000A24120CA8306D03120738120DC2120EAD
:10155800A8120A24120C97306D03120796120DC2B6
:10156800120ECD120A24120CA8306D031207F312C2
:101578000DC2120F44120A2412093E120C97120DC2
:10158800C2120F69120942120A2430692F206B2CEB
:1015980085676485676585636C756D0179187A0C54
:1015A800C3E533994009C269D26A8A350215C4C3B2
:1015B800E55F9401400302151D02161E306A1B20C8
:1015C8006B18E535147004C26AA111F535C3E55FDF
:1015D8009401400302151D02161E753600C3E5620C
:1015E8009401400985676585636C756D01C3E56283
:1015F80078FA985021307404E52A601A78F0306B34
:10160800058567647820C3E541985002A11D053619
:10161800E55F6002C121753600C2AF120FDE788720
:10162800E6FE7602115C7887EEF6E4F522F523F5FE
:1016380024F525F526F568C268D2AF120553120FB6
:10164800DE307406E52A700221FB788DE6C394012A
:10165800400241CF61FA901A0D78201216E2E52077
:10166800B4A50CA31216E2E520B45A0302168012A0
:101678000FF31216A002169F901A0378807B0A12A5
:1016880016E2A308DBF9901A0F788C7B181216E281
:10169800A308DBF9901A2722C2AF1217211216FBF2
:1016A800901A00740E1216E7A374041216E7A374B6
:1016B800141216E7901A0378807B0A1216E6A3081C
:1016C800DBF9901A0F788C7B181216E6A308DBF961
:1016D800121734121712901A2722E493F622E643BF
:1016E8008F01538FFD75EF0275B7A575B7F1F053EC
:1016F8008FFE22438F02438F0175EF0275B7A575E0
:10170800B7F1901A0DF0538FFC22901A0D74A5D1E1
:10171800E7901A0E745AD1E7227A3079D07820905F
:101728001A40D1E2E520F709A3DAF7227A3079D016
:10173800901A40E7D1E709A3DAF922AB77A878BB7A
:1017480001027980BB02027981BB03027982BB0462
:10175800027994BB05027983BB06027986BB07022E
:101768007992BB08027987BB0902799CBB0A027986
:1017780088BB0B027989E8F7227C0512056CDCFB33
:1017880022C2AF12057C12058312058A1205911236
:10179800055D12057C12058312058A120591120552
:1017A8005D12057C12058312058A120591D2AF22BB
:1017B800C2AF12059112058A12058312057C120523
:1017C8005D12059112058A12058312057C12055DCA
:1017D80012059112058A12058312057CD2AF22AE3A
:1017E80077AF78C2AF12057C12057C12057C120512
:1017F8005DDEF212059112055DDFF8D2AF221217F5
:10180800891217811217817577017578017579002A
:101818001217E77C05AD5F12056CC3ED955F70F597
:10182800C3E55F9401400AC3E55F94FF403702189F
:101838004A1217431216A0121789C2AF75EF121277
:101848001781DCD10579C3E5799403500280C11270
:1018580017810578E5771490009F93F808C3E57819
:0E18680098500280A81217811217810577C3CD
:10187600E577940C50028094120FF31216A0C2AFB3
:0618860075EF121217813C
:0319FD0002115D77
:101A00000E041407070104FFFF0A020101A55A0191
:101A100000B4FFFFFF03FF01FF25D078C804FF01DA
:081A200000FF0A010100FFFFB5
:101A400023536B7977616C6B6572323041232020B0
:101A500023424C48454C4923463333302320202031
:101A60002020202020202020202020202020202076
:101C0000C2AFC2D353D9BF7581C043B20343FF8073
:101C1000752438752503B1C975EF0275E24043F1AB
:101C20002053A4DF75D400D2857DFA780379E67C51
:101C300010752200752300901DD67B0675249875BB
:101C400025013085028142208508D8FBD9F9DCF7CF
:101C500081B4308508D8FBD9F9DCF781B4B189E4C7
:101C600093A3C39A6004DDC381B4DBDBB17B600264
:101C7000812B7B08E493FAA3B15CDBF87A30B15C8A
:101C8000752200752300B17BEAFCEBFDC3ED94FEE9
:101C9000400EB17B8A278B28ED30E0048A828B834B
:101CA000B17B7AC270D8C3ED94FE601350CEBD00F4
:101CB00025EC60097520007521FF0200008100A855
:101CC00027A9280809D804D90281D3B17FEA89AAB3
:101CD000F281C50D81A0C3ED94035049EDA2E092BD
:101CE000007AC5C3E5829400E583941C50902000DF
:101CF00010438F02438F0175B7A575B7F1F030001F
:101D00001FA827A9280809438F01538FFDD804D99C
:101D100002A12089AAE275B7A575B7F1F0A3A10DBC
:101D2000538FFC817C7AC1BD030CE493A3FAB140CC
:101D3000DCF8B138817C817EAA22AB23B15CEBFA5E
:101D4000EA6222752608C3E52313F523E52213F57D
:101D50002250066323A0632201D526EAB1C9B1C986
:101D600075260AEAF4200102D285300102C285B14B
:101D7000C9C3134002C201D526EB22B17FEAFB2082
:101D80008502A17F308502A184752608AE24AF2587
:101D9000C3EF13FFEE13FEB1CDB1C9C3EA13308513
:101DA000024480FA30E703632201C3E52313F523DD
:101DB000E52213F52250066323A0632201D526D91C
:101DC000E52265236523F52222AE24AF250E0FDE22
:101DD000FEDFFCD20122424C48656C693437316326
:041DE000F3300601D5
:00000001FF
